 services_test

 Timestamp is 4be8ceb2 (Tue May 11 12:27:46 2010)

 Preferred load address is 00010000

 Start         Length     Name                   Class
 0001:00000000 00000004H .CRT$XCA                CODE
 0001:00000004 00000004H .CRT$XCZ                CODE
 0001:00000008 00000004H .CRT$XIA                CODE
 0001:0000000c 00000004H .CRT$XIZ                CODE
 0001:00000010 00000004H .CRT$XPA                CODE
 0001:00000014 00000004H .CRT$XPZ                CODE
 0001:00000018 00000004H .CRT$XTA                CODE
 0001:0000001c 00000004H .CRT$XTZ                CODE
 0001:00000020 00000bd4H .rdata                  CODE
 0001:00000bf4 0000002aH .rdata$debug            CODE
 0001:00000c20 000016d8H .text                   CODE
 0001:000022f8 00000018H .xdata                  CODE
 0001:00002310 00000028H .idata$2                CODE
 0001:00002338 00000014H .idata$3                CODE
 0001:0000234c 000000c8H .idata$4                CODE
 0001:00002414 00000120H .idata$6                CODE
 0001:00002534 00000000H .edata                  CODE
 0002:00000000 000000c8H .idata$5                DATA
 0002:000000c8 00000008H .data                   DATA
 0002:000000d0 00000010H .bss                    DATA
 0003:00000000 00000080H .pdata                  DATA

  Address         Publics by Value              Rva+Base       Lib:Object

 0000:00000000       ___safe_se_handler_table   00000000     <absolute>
 0000:00000000       ___safe_se_handler_count   00000000     <absolute>
 0001:00000000       __xc_a                     00011000     corelib0:crt0init.obj
 0001:00000004       __xc_z                     00011004     corelib0:crt0init.obj
 0001:00000008       __xi_a                     00011008     corelib0:crt0init.obj
 0001:0000000c       __xi_z                     0001100c     corelib0:crt0init.obj
 0001:00000010       __xp_a                     00011010     corelib0:crt0init.obj
 0001:00000014       __xp_z                     00011014     corelib0:crt0init.obj
 0001:00000018       __xt_a                     00011018     corelib0:crt0init.obj
 0001:0000001c       __xt_z                     0001101c     corelib0:crt0init.obj
 0001:0000003c       ??_C@_0BD@FOHFKAOE@INVALID?5ERROR?5CODE?$AA@ 0001103c     services_test.obj
 0001:00000050       ??_C@_09KMCHPOPM@PVRSRV_OK?$AA@ 00011050     services_test.obj
 0001:0000005c       ??_C@_0BF@KHEAJDEG@PVRSRV_ERROR_GENERIC?$AA@ 0001105c     services_test.obj
 0001:00000074       ??_C@_0BL@BOENCAIM@PVRSRV_ERROR_OUT_OF_MEMORY?$AA@ 00011074     services_test.obj
 0001:00000090       ??_C@_0BO@BBFKIBH@PVRSRV_ERROR_TOO_MANY_BUFFERS?$AA@ 00011090     services_test.obj
 0001:000000b0       ??_C@_0BO@EGNEIFEA@PVRSRV_ERROR_SYMBOL_NOT_FOUND?$AA@ 000110b0     services_test.obj
 0001:000000d0       ??_C@_0BL@BKMGFOLH@PVRSRV_ERROR_OUT_OF_HSPACE?$AA@ 000110d0     services_test.obj
 0001:000000ec       ??_C@_0BM@LGNAOM@PVRSRV_ERROR_INVALID_PARAMS?$AA@ 000110ec     services_test.obj
 0001:00000108       ??_C@_0BN@MGJEIKFE@PVRSRV_ERROR_TILE_MAP_FAILED?$AA@ 00011108     services_test.obj
 0001:00000128       ??_C@_0BK@JHPIKHJG@PVRSRV_ERROR_INIT_FAILURE?$AA@ 00011128     services_test.obj
 0001:00000144       ??_C@_0CE@POPMCOCG@PVRSRV_ERROR_CANT_REGISTER_CALLB@ 00011144     services_test.obj
 0001:00000168       ??_C@_0BM@COIEDMNF@PVRSRV_ERROR_INVALID_DEVICE?$AA@ 00011168     services_test.obj
 0001:00000184       ??_C@_0BH@OEOFFCIM@PVRSRV_ERROR_NOT_OWNER?$AA@ 00011184     services_test.obj
 0001:0000019c       ??_C@_0BJ@PHFCJIBD@PVRSRV_ERROR_BAD_MAPPING?$AA@ 0001119c     services_test.obj
 0001:000001b8       ??_C@_0BF@KGIMOMJE@PVRSRV_ERROR_TIMEOUT?$AA@ 000111b8     services_test.obj
 0001:000001d0       ??_C@_0BI@CDPBDDFH@PVRSRV_ERROR_NO_PRIMARY?$AA@ 000111d0     services_test.obj
 0001:000001e8       ??_C@_0BP@FMELGOJO@PVRSRV_ERROR_FLIP_CHAIN_EXISTS?$AA@ 000111e8     services_test.obj
 0001:00000208       ??_C@_0BN@JMHJCLJP@ERROR_CANNOT_ACQUIRE_SYSDATA?$AA@ 00011208     services_test.obj
 0001:00000228       ??_C@_0BL@JPEIBKNH@PVRSRV_ERROR_SCENE_INVALID?$AA@ 00011228     services_test.obj
 0001:00000244       ??_C@_0BK@JAAFMMBM@PVRSRV_ERROR_STREAM_ERROR?$AA@ 00011244     services_test.obj
 0001:00000260       ??_C@_0DP@FHJOPEMA@PVRSRV_ERROR_INVALID_INTERRUPTPV@ 00011260     services_test.obj
 0001:000002a0       ??_C@_0BP@PFBLKCEO@PVRSRV_ERROR_CMD_NOT_PROCESSED?$AA@ 000112a0     services_test.obj
 0001:000002c0       ??_C@_0BJ@PHLIKBPN@PVRSRV_ERROR_CMD_TOO_BIG?$AA@ 000112c0     services_test.obj
 0001:000002dc       ??_C@_0CE@FHHHLEGE@PVRSRV_ERROR_DEVICE_REGISTER_FAI@ 000112dc     services_test.obj
 0001:00000300       ??_C@_0BI@JBKNPCOM@PVRSRV_ERROR_FIFO_SPACE?$AA@ 00011300     services_test.obj
 0001:00000318       ??_C@_0BJ@IIGHNIEG@PVRSRV_ERROR_TA_RECOVERY?$AA@ 00011318     services_test.obj
 0001:00000334       ??_C@_0BJ@IMBALOKG@PVRSRV_DEVICE_ID_UNKNOWN?$AA@ 00011334     services_test.obj
 0001:00000350       ??_C@_0BH@OGEGGGCD@PVRSRV_DEVICE_ID_MSVDX?$AA@ 00011350     services_test.obj
 0001:00000368       ??_C@_0BF@BBCLGMON@PVRSRV_DEVICE_ID_SGX?$AA@ 00011368     services_test.obj
 0001:00000380       ??_C@_0CD@BDGFMHBG@PVRSRV_DEVICE_TYPE_EXT?5?$CI3rd?5Part@ 00011380     services_test.obj
 0001:000003a4       ??_C@_0BE@GEDKFGMC@Not?5recognised?50x?$CFx?$AA@ 000113a4     services_test.obj
 0001:000003b8       ??_C@_0BI@ICLDLMDM@?4?4?4?4?5ui32ProcessID?3?$CFlu?6?$AA@ 000113b8     services_test.obj
 0001:000003d0       ??_C@_0CA@OBOKIFIC@Reached?5exit?5point?5?$CFu?4?5Exiting?4?$AA@ 000113d0     services_test.obj
 0001:000003f0       ??_C@_0M@FBGHFOFL@?5FAIL?5?9?5?$CFs?6?$AA@ 000113f0     services_test.obj
 0001:000003fc       ??_C@_06HEMPAKAM@?5FAIL?6?$AA@ 000113fc     services_test.obj
 0001:00000404       ??_C@_0DH@PINPAELL@?9?9?9?9?9?9?9?9?9?9?9?9?9?9?9?9?9?9?9?9?9End?5loop?5?$CFd@ 00011404     services_test.obj
 0001:0000043c       ??_C@_0BD@NOILHFAN@PVRSRVDisconnect?3?6?$AA@ 0001143c     services_test.obj
 0001:00000450       ??_C@_0BH@LMCBNGLN@SGXReleaseClientInfo?3?6?$AA@ 00011450     services_test.obj
 0001:00000468       ??_C@_0CF@DBFHMBAF@Display?5Class?5API?3?5close?5the?5dev@ 00011468     services_test.obj
 0001:00000490       ??_C@_0CM@LDEJMMMA@Attempt?5to?5destroy?5memory?5contex@ 00011490     services_test.obj
 0001:000004bc       ??_C@_0DD@GODBIEMM@Display?5Class?5API?3?5unmap?5display@ 000114bc     services_test.obj
 0001:000004f0       ??_C@_0CE@CHFCNMEA@Attempt?5to?5destroy?5render?5contex@ 000114f0     services_test.obj
 0001:00000514       ??_C@_0O@COCNECFL@DDK?5version?3?6?$AA@ 00011514     services_test.obj
 0001:00000524       ??_C@_0BB@EOMOJBAE@?$CFld?4?$CFld?4?$CFld?4?$CFld?6?$AA@ 00011524     services_test.obj
 0001:00000538       ??_C@_0BI@ODLJPBGI@DDK?5version?5string?3?5?$CFs?6?$AA@ 00011538     services_test.obj
 0001:00000550       ??_C@_0CC@FHJCCNNC@Attempt?5to?5remove?5render?5target?3@ 00011550     services_test.obj
 0001:00000574       ??_C@_02DKCKIIND@?$CFs?$AA@ 00011574     services_test.obj
 0001:00000578       ??_C@_0BI@JIPAPGGA@Gather?5some?5mem?5stats?3?6?$AA@ 00011578     services_test.obj
 0001:00000590       ??_C@_0CH@PLJFMKGN@Attempt?5to?5add?5render?5target?5for@ 00011590     services_test.obj
 0001:000005b8       ??_C@_0CO@LLJKCOKB@Attempt?5to?5create?5rendering?5cont@ 000115b8     services_test.obj
 0001:000005e8       ??_C@_0CP@IFAFGPME@Display?5Class?5API?3?5map?5display?5s@ 000115e8     services_test.obj
 0001:00000618       ??_C@_0EK@BPNJOJAB@?4?4?4?4?5Shared?5heap?5?$CFlu?5?9?5HeapID?30x@ 00011618     services_test.obj
 0001:00000664       ??_C@_0DE@BODOPOHG@Display?5Class?5API?3?5get?5the?5syste@ 00011664     services_test.obj
 0001:00000698       ??_C@_0ED@NNKEOJPF@?4?4?4?4?5Display?5dimensions?5?$CFlu?5?9?5By@ 00011698     services_test.obj
 0001:000006dc       ??_C@_0DB@DPDHNDGF@Display?5Class?5API?3?5enumerate?5dis@ 000116dc     services_test.obj
 0001:00000710       ??_C@_0CK@PAKBMFJN@?4?4?4?4?5Display?5format?5?$CFlu?5?9?5Pixelf@ 00011710     services_test.obj
 0001:0000073c       ??_C@_0O@GDPIEJBG@?4?4?4?4?5Name?3?$CFs?6?$AA@ 0001173c     services_test.obj
 0001:0000074c       ??_C@_0BI@BLGHILNJ@?4?4?4?4?5MaxSwapChains?3?$CFlu?6?$AA@ 0001174c     services_test.obj
 0001:00000764       ??_C@_0BO@POAFDAJE@?4?4?4?4?5MaxSwapChainBuffers?3?$CFlu?6?$AA@ 00011764     services_test.obj
 0001:00000784       ??_C@_0BK@CPCAOBID@?4?4?4?4?5MinSwapInterval?3?$CFlu?6?$AA@ 00011784     services_test.obj
 0001:000007a0       ??_C@_0BK@DMGFAHCI@?4?4?4?4?5MaxSwapInterval?3?$CFlu?6?$AA@ 000117a0     services_test.obj
 0001:000007bc       ??_C@_0CO@GIPBIACE@Display?5Class?5API?3?5enumerate?5dis@ 000117bc     services_test.obj
 0001:000007ec       ??_C@_0CF@FMDFFMKC@Display?5Class?5API?3?5Get?5display?5i@ 000117ec     services_test.obj
 0001:00000814       ??_C@_0CA@DAONOMAK@Display?5Class?5API?3?5open?5device?6?$AA@ 00011814     services_test.obj
 0001:00000834       ??_C@_0CL@DNLHEBLI@Attempt?5to?5create?5memory?5context@ 00011834     services_test.obj
 0001:00000860       ??_C@_0CA@DGGJNKGO@?5Test?5Memory?5Allocation?5FAILED?6?$AA@ 00011860     services_test.obj
 0001:00000880       ??_C@_0DM@CIPNLPOO@PVRSRVEnumerateDeviceClass?$CI?$CJ?5ret@ 00011880     services_test.obj
 0001:000008bc       ??_C@_0CG@MMBLEMBO@Display?5Class?5API?3?5enumerate?5dev@ 000118bc     services_test.obj
 0001:000008e4       ??_C@_0BJ@NLALCGOE@Getting?5SGX?5Client?5info?6?$AA@ 000118e4     services_test.obj
 0001:00000900       ??_C@_0BP@IDIGABKI@Attempt?5to?5acquire?5device?5?$CFd?3?6?$AA@ 00011900     services_test.obj
 0001:00000920       ??_C@_0BH@PPGIPGOP@?5?5?5?5?5?5?5?5?5?5?5?5?$CF04d?5?5?5?5?$HM?5?$AA@ 00011920     services_test.obj
 0001:00000938       ??_C@_01EEMJAFIK@?6?$AA@   00011938     services_test.obj
 0001:0000093c       ??_C@_0BK@GEDDINJE@?4?4?4?4?5Reported?5?$CFu?5devices?6?$AA@ 0001193c     services_test.obj
 0001:00000958       ??_C@_0CD@INKLJIDI@?4?4?4?4?5Device?5Number?5?5?$HM?5Device?5Typ@ 00011958     services_test.obj
 0001:0000097c       ??_C@_0DE@KAFOOJDI@Get?5number?5of?5devices?5from?5PVRSR@ 0001197c     services_test.obj
 0001:000009b0       ??_C@_0EA@LNIAFGAD@Try?5calling?5PVRSRVEnumerateDevic@ 000119b0     services_test.obj
 0001:000009f0       ??_C@_04LNELOFCG@?5OK?6?$AA@ 000119f0     services_test.obj
 0001:000009f8       ??_C@_0CL@KFFMIBHA@Call?5PVRSRVConnect?5with?5a?5valid?5@ 000119f8     services_test.obj
 0001:00000a24       ??_C@_0DH@PPPHAACG@?9?9?9?9?9?9?9?9?9?9?9?9?9?9?9?9?9?9?9?9?9?9?9?5Start?5?9?9@ 00011a24     services_test.obj
 0001:00000a5c       ??_C@_0DF@NBHKCIFP@Try?5calling?5PVRSRVConnect?5with?5a@ 00011a5c     services_test.obj
 0001:00000a98       ??_C@_1KE@BDGMONOJ@?$AAH?$AA?3?$AA?2?$AAW?$AAI?$AAN?$AAC?$AAE?$AA6?$AA0?$AA0?$AA?2?$AAP?$AAL?$AAA?$AAT?$AAF?$AAO?$AAR?$AAM?$AA?2?$AAS?$AAM?$AAD?$AAK?$AAV?$AA2?$AA1?$AA0?$AA?2?$AAS?$AAR@ 00011a98     wince_unittests.obj
 0001:00000b3c       ??_C@_1CI@OHCJFJPM@?$AAE?$AAR?$AAR?$AAO?$AAR?$AA?3?$AA?5?$AA?$CF?$AAs?$AA?5?$AAl?$AAi?$AAn?$AAe?$AA?5?$AA?$CF?$AAd?$AA?3?$AA?5?$AA?$AA@ 00011b3c     wince_unittests.obj
 0001:00000b64       ??_C@_1CK@MPGKAOE@?$AA?$CI?$AAe?$AAr?$AAr?$AAo?$AAr?$AA?5?$AAc?$AAo?$AAd?$AAe?$AA?3?$AA?5?$AA?$CF?$AAd?$AA?$CJ?$AA?3?$AA?5?$AA?$CF?$AAs?$AA?$AA@ 00011b64     wince_unittests.obj
 0001:00000b90       ??_C@_1M@DMCDIEDK@?$AAP?$AAK?$AAM?$AA1?$AA?3?$AA?$AA@ 00011b90     wince_unittests.obj
 0001:00000b9c       ??_C@_0L@GPAGIAIC@?9disablepm?$AA@ 00011b9c     wince_unittests.obj
 0001:00000ba8       ??_C@_1M@ILHOPKA@?$AAE?$AAr?$AAr?$AAo?$AAr?$AA?$AA@ 00011ba8     wince_unittests.obj
 0001:00000bb4       ??_C@_1DG@PCJNAHOH@?$AAF?$AAa?$AAi?$AAl?$AAe?$AAd?$AA?5?$AAt?$AAo?$AA?5?$AAg?$AAe?$AAt?$AA?5?$AAm?$AAo?$AAn?$AAi?$AAt?$AAo?$AAr?$AA?5?$AAi?$AAn?$AAf?$AAo?$AA?$AA@ 00011bb4     wince_unittests.obj
 0001:00000bec       ??_C@_07FBLHGNAH@app?4exe?$AA@ 00011bec     wince_unittests.obj
 0001:00000d7c       print_dev_type             00011d7c f   services_test.obj
 0001:00000ddc       main                       00011ddc f   services_test.obj
 0001:00001a04       WinMain                    00012a04 f   wince_unittests.obj
 0001:00001ca8       ReleasePowerRequirement    00012ca8 f   coredll:COREDLL.dll
 0001:00001cb8       NKDbgPrintfW               00012cb8 f   coredll:COREDLL.dll
 0001:00001cc8       FormatMessageW             00012cc8 f   coredll:COREDLL.dll
 0001:00001cd8       GetLastError               00012cd8 f   coredll:COREDLL.dll
 0001:00001ce8       SetPowerRequirement        00012ce8 f   coredll:COREDLL.dll
 0001:00001cf8       WideCharToMultiByte        00012cf8 f   coredll:COREDLL.dll
 0001:00001d08       SetCursorPos               00012d08 f   coredll:COREDLL.dll
 0001:00001d18       GetCursorPos               00012d18 f   coredll:COREDLL.dll
 0001:00001d28       MessageBoxW                00012d28 f   coredll:COREDLL.dll
 0001:00001d38       GetMonitorInfo             00012d38 f   coredll:COREDLL.dll
 0001:00001d48       MonitorFromPoint           00012d48 f   coredll:COREDLL.dll
 0001:00001d58       PVRSRVDisconnect           00012d58 f   srvclum:SRVCLUM.dll
 0001:00001d68       SGXReleaseClientInfo       00012d68 f   srvclum:SRVCLUM.dll
 0001:00001d78       PVRSRVCloseDCDevice        00012d78 f   srvclum:SRVCLUM.dll
 0001:00001d88       PVRSRVDestroyDeviceMemContext 00012d88 f   srvclum:SRVCLUM.dll
 0001:00001d98       PVRSRVUnmapDeviceClassMemory 00012d98 f   srvclum:SRVCLUM.dll
 0001:00001da8       SGXDestroyRenderContext    00012da8 f   srvclum:SRVCLUM.dll
 0001:00001db8       SGXRemoveRenderTarget      00012db8 f   srvclum:SRVCLUM.dll
 0001:00001dc8       PVRSRVFreeUserModeMem      00012dc8 f   srvclum:SRVCLUM.dll
 0001:00001dd8       PVRSRVGetMiscInfo          00012dd8 f   srvclum:SRVCLUM.dll
 0001:00001de8       PVRSRVAllocUserModeMem     00012de8 f   srvclum:SRVCLUM.dll
 0001:00001df8       SGXAddRenderTarget         00012df8 f   srvclum:SRVCLUM.dll
 0001:00001e08       SGXCreateRenderContext     00012e08 f   srvclum:SRVCLUM.dll
 0001:00001e18       PVRSRVMapDeviceClassMemory 00012e18 f   srvclum:SRVCLUM.dll
 0001:00001e28       PVRSRVGetDCSystemBuffer    00012e28 f   srvclum:SRVCLUM.dll
 0001:00001e38       PVRSRVEnumDCDims           00012e38 f   srvclum:SRVCLUM.dll
 0001:00001e48       PVRSRVEnumDCFormats        00012e48 f   srvclum:SRVCLUM.dll
 0001:00001e58       PVRSRVGetDCInfo            00012e58 f   srvclum:SRVCLUM.dll
 0001:00001e68       PVRSRVOpenDCDevice         00012e68 f   srvclum:SRVCLUM.dll
 0001:00001e78       PVRSRVCreateDeviceMemContext 00012e78 f   srvclum:SRVCLUM.dll
 0001:00001e88       PVRSRVEnumerateDeviceClass 00012e88 f   srvclum:SRVCLUM.dll
 0001:00001e98       SGXGetClientInfo           00012e98 f   srvclum:SRVCLUM.dll
 0001:00001ea8       PVRSRVAcquireDeviceData    00012ea8 f   srvclum:SRVCLUM.dll
 0001:00001eb8       PVRSRVEnumerateDevices     00012eb8 f   srvclum:SRVCLUM.dll
 0001:00001ec8       PVRSRVConnect              00012ec8 f   srvclum:SRVCLUM.dll
 0001:00001f58       WinMainCRTStartup          00012f58 f   corelib0:pegwmain.obj
 0001:00002054       exit                       00013054 f   corelib0:cexit.obj
 0001:0000206c       _exit                      0001306c f   corelib0:cexit.obj
 0001:000020ac       __GSHandlerCheckCommon     000130ac f   corelib0:gshandler.obj
 0001:000020e8       __GSHandlerCheck           000130e8 f   corelib0:gshandler.obj
 0001:0000210c       __security_init_cookie     0001310c f   corelib0:seccinit.obj
 0001:00002168       __security_check_cookie    00013168 f   corelib0:armsecgs.obj
 0001:0000217c       __gsfailure                0001317c f   corelib0:armsecgs.obj
 0001:000021c0       _initterm                  000131c0 f   corelib0:crt0dat.obj
 0001:000021f4       _cinit                     000131f4 f   corelib0:crt0dat.obj
 0001:00002228       printf                     00013228 f   corelib1:COREDLL.dll
 0001:00002238       free                       00013238 f   corelib1:COREDLL.dll
 0001:00002248       malloc                     00013248 f   corelib1:COREDLL.dll
 0001:00002258       atol                       00013258 f   corelib1:COREDLL.dll
 0001:00002268       _stricmp                   00013268 f   corelib1:COREDLL.dll
 0001:00002278       _isctype                   00013278 f   corelib1:COREDLL.dll
 0001:00002288       wcslen                     00013288 f   corelib1:COREDLL.dll
 0001:00002298       memset                     00013298 f   corelib1:COREDLL.dll
 0001:000022a8       _XcptFilter                000132a8 f   corelib1:COREDLL.dll
 0001:000022b8       __C_specific_handler       000132b8 f   corelib1:COREDLL.dll
 0001:000022c8       __security_gen_cookie2     000132c8 f   corelib1:COREDLL.dll
 0001:000022d8       __report_gsfailure         000132d8 f   corelib1:COREDLL.dll
 0001:000022e8       TerminateProcess           000132e8 f   coredll:COREDLL.dll
 0001:00002310       __IMPORT_DESCRIPTOR_COREDLL 00013310     coredll:COREDLL.dll
 0001:00002324       __IMPORT_DESCRIPTOR_SRVCLUM 00013324     srvclum:SRVCLUM.dll
 0001:00002338       __NULL_IMPORT_DESCRIPTOR   00013338     coredll:COREDLL.dll
 0002:00000000       __imp_ReleasePowerRequirement 00014000     coredll:COREDLL.dll
 0002:00000004       __imp_NKDbgPrintfW         00014004     coredll:COREDLL.dll
 0002:00000008       __imp_FormatMessageW       00014008     coredll:COREDLL.dll
 0002:0000000c       __imp_GetLastError         0001400c     coredll:COREDLL.dll
 0002:00000010       __imp_SetPowerRequirement  00014010     coredll:COREDLL.dll
 0002:00000014       __imp_WideCharToMultiByte  00014014     coredll:COREDLL.dll
 0002:00000018       __imp_SetCursorPos         00014018     coredll:COREDLL.dll
 0002:0000001c       __imp_GetCursorPos         0001401c     coredll:COREDLL.dll
 0002:00000020       __imp_MessageBoxW          00014020     coredll:COREDLL.dll
 0002:00000024       __imp_GetMonitorInfo       00014024     coredll:COREDLL.dll
 0002:00000028       __imp_MonitorFromPoint     00014028     coredll:COREDLL.dll
 0002:0000002c       __imp___report_gsfailure   0001402c     corelib1:COREDLL.dll
 0002:00000030       __imp___security_gen_cookie2 00014030     corelib1:COREDLL.dll
 0002:00000034       __imp___C_specific_handler 00014034     corelib1:COREDLL.dll
 0002:00000038       __imp__XcptFilter          00014038     corelib1:COREDLL.dll
 0002:0000003c       __imp_memset               0001403c     corelib1:COREDLL.dll
 0002:00000040       __imp_wcslen               00014040     corelib1:COREDLL.dll
 0002:00000044       __imp__isctype             00014044     corelib1:COREDLL.dll
 0002:00000048       __imp__stricmp             00014048     corelib1:COREDLL.dll
 0002:0000004c       __imp_atol                 0001404c     corelib1:COREDLL.dll
 0002:00000050       __imp_TerminateProcess     00014050     coredll:COREDLL.dll
 0002:00000054       __imp_malloc               00014054     corelib1:COREDLL.dll
 0002:00000058       __imp_free                 00014058     corelib1:COREDLL.dll
 0002:0000005c       __imp_printf               0001405c     corelib1:COREDLL.dll
 0002:00000060       \177COREDLL_NULL_THUNK_DATA 00014060     coredll:COREDLL.dll
 0002:00000064       __imp_PVRSRVGetDCInfo      00014064     srvclum:SRVCLUM.dll
 0002:00000068       __imp_PVRSRVOpenDCDevice   00014068     srvclum:SRVCLUM.dll
 0002:0000006c       __imp_PVRSRVCreateDeviceMemContext 0001406c     srvclum:SRVCLUM.dll
 0002:00000070       __imp_PVRSRVEnumerateDeviceClass 00014070     srvclum:SRVCLUM.dll
 0002:00000074       __imp_SGXGetClientInfo     00014074     srvclum:SRVCLUM.dll
 0002:00000078       __imp_PVRSRVAcquireDeviceData 00014078     srvclum:SRVCLUM.dll
 0002:0000007c       __imp_PVRSRVEnumerateDevices 0001407c     srvclum:SRVCLUM.dll
 0002:00000080       __imp_PVRSRVConnect        00014080     srvclum:SRVCLUM.dll
 0002:00000084       __imp_PVRSRVEnumDCFormats  00014084     srvclum:SRVCLUM.dll
 0002:00000088       __imp_PVRSRVEnumDCDims     00014088     srvclum:SRVCLUM.dll
 0002:0000008c       __imp_PVRSRVGetDCSystemBuffer 0001408c     srvclum:SRVCLUM.dll
 0002:00000090       __imp_SGXCreateRenderContext 00014090     srvclum:SRVCLUM.dll
 0002:00000094       __imp_SGXAddRenderTarget   00014094     srvclum:SRVCLUM.dll
 0002:00000098       __imp_PVRSRVAllocUserModeMem 00014098     srvclum:SRVCLUM.dll
 0002:0000009c       __imp_PVRSRVGetMiscInfo    0001409c     srvclum:SRVCLUM.dll
 0002:000000a0       __imp_PVRSRVFreeUserModeMem 000140a0     srvclum:SRVCLUM.dll
 0002:000000a4       __imp_SGXRemoveRenderTarget 000140a4     srvclum:SRVCLUM.dll
 0002:000000a8       __imp_SGXDestroyRenderContext 000140a8     srvclum:SRVCLUM.dll
 0002:000000ac       __imp_PVRSRVUnmapDeviceClassMemory 000140ac     srvclum:SRVCLUM.dll
 0002:000000b0       __imp_PVRSRVDestroyDeviceMemContext 000140b0     srvclum:SRVCLUM.dll
 0002:000000b4       __imp_PVRSRVCloseDCDevice  000140b4     srvclum:SRVCLUM.dll
 0002:000000b8       __imp_SGXReleaseClientInfo 000140b8     srvclum:SRVCLUM.dll
 0002:000000bc       __imp_PVRSRVDisconnect     000140bc     srvclum:SRVCLUM.dll
 0002:000000c0       __imp_PVRSRVMapDeviceClassMemory 000140c0     srvclum:SRVCLUM.dll
 0002:000000c4       \177SRVCLUM_NULL_THUNK_DATA 000140c4     srvclum:SRVCLUM.dll
 0002:000000c8       __security_cookie          000140c8     corelib0:seccinit.obj
 0002:000000cc       __security_cookie_complement 000140cc     corelib0:seccinit.obj
 0002:000000d0       pfnRegisteredWndProc       000140d0     wince_unittests.obj
 0002:000000d4       _exitflag                  000140d4     corelib0:cexit.obj
 0002:000000d8       __onexitend                000140d8     <common>
 0002:000000dc       __onexitbegin              000140dc     <common>

 entry point at        0001:00001f58

 Static symbols

 0001:00000c20       GetString                  00011c20 f   services_test.obj
 0001:00001ee0       WinMainCRTStartupHelper    00012ee0 f   corelib0:pegwmain.obj
 0001:00001f8c       doexit                     00012f8c f   corelib0:cexit.obj
